:020000040800F2
:1000000000090020F50400086928000821280008DC
:10001000492800082128000841280008F7040008A2
:10002000F7040008F7040008F7040008493800083E
:10003000F7040008F7040008F7040008F7040008B4
:10004000F7040008F7040008F7040008F7040008A4
:10005000F7040008F7040008BD450008E54500085E
:100060000D460008354600085D460008F704000804
:10007000F7040008F7040008F7040008F704000874
:10008000F7040008F7040008F7040008F704000864
:10009000F704000801280008112800088546000818
:1000A000F7040008F7040008F7040008F704000844
:1000B00059470008F7040008F7040008F70400088F
:1000C000F7040008F7040008F7040008F704000824
:1000D000F7040008F7040008F7040008F704000814
:1000E000E9460008F7040008F7040008F7040008D0
:1000F000F7040008F7040008F7040008F7040008F4
:10010000F7040008F7040008F7040008F7040008E3
:10011000F7040008F7040008F7040008F7040008D3
:10012000F7040008F7040008F7040008F7040008C3
:10013000F7040008F7040008F7040008F7040008B3
:10014000F7040008F7040008F7040008F7040008A3
:10015000F7040008F7040008F7040008F704000893
:10016000F7040008F7040008F7040008F704000883
:10017000F7040008F7040008F7040008F704000873
:10018000F7040008F7040008F7040008F704000863
:10019000F7040008F7040008F7040008F704000853
:1001A000F7040008F7040008F7040008F704000843
:1001B000F7040008F7040008F7040008F704000833
:1001C000F7040008F7040008F7040008F704000823
:1001D000F7040008F7040008F7040008F704000813
:1001E0007112000800000000000000000000000084
:1001F00053B94AB9002908BF00281CBF4FF0FF318E
:100200004FF0FF3000F074B9ADF1080C6DE904CE89
:1002100000F006F8DDF804E0DDE9022304B07047E1
:100220002DE9F047089D04468E46002B4DD18A42A9
:10023000944669D9B2FA82F252B101FA02F3C2F1DC
:10024000200120FA01F10CFA02FC41EA030E94406D
:100250004FEA1C48210CBEFBF8F61FFA8CF708FB8E
:1002600016E341EA034306FB07F199420AD91CEB66
:10027000030306F1FF3080F01F81994240F21C8198
:10028000023E63445B1AA4B2B3FBF8F008FB1033E0
:1002900044EA034400FB07F7A7420AD91CEB040415
:1002A00000F1FF3380F00A81A74240F207816444E5
:1002B000023840EA0640E41B00261DB1D44000236A
:1002C000C5E900433146BDE8F0878B4209D9002DCE
:1002D00000F0EF800026C5E9000130463146BDE858
:1002E000F087B3FA83F6002E4AD18B4202D38242C2
:1002F00000F2F980841A61EB030301209E46002D71
:10030000E0D0C5E9004EDDE702B9FFDEB2FA82F2C5
:10031000002A40F09280A1EB0C014FEA1C471FFA23
:100320008CFE0126200CB1FBF7F307FB131140EA0A
:1003300001410EFB03F0884208D91CEB010103F1D7
:10034000FF3802D2884200F2CB804346091AA4B299
:10035000B1FBF7F007FB101144EA01440EFB00FE6D
:10036000A64508D91CEB040400F1FF3102D2A645D2
:1003700000F2BB800846A4EB0E0440EA03409CE771
:10038000C6F12007B34022FA07FC4CEA030C20FA1E
:1003900007F401FA06F31C43F9404FEA1C4900FA3E
:1003A00006F3B1FBF9F8200C1FFA8CFE09FB1811BB
:1003B00040EA014108FB0EF0884202FA06F20BD92E
:1003C0001CEB010108F1FF3A80F08880884240F27E
:1003D0008580A8F102086144091AA4B2B1FBF9F0C2
:1003E00009FB101144EA014100FB0EFE8E4508D9BD
:1003F0001CEB010100F1FF346CD28E456AD9023842
:10040000614440EA0840A0FB0294A1EB0E01A14226
:10041000C846A64656D353D05DB1B3EB080261EB94
:100420000E0101FA07F722FA06F3F1401F43C5E96E
:10043000007100263146BDE8F087C2F12003D840A4
:100440000CFA02FC21FA03F3914001434FEA1C47E6
:100450001FFA8CFEB3FBF7F007FB10360B0C43EAD8
:10046000064300FB0EF69E4204FA02F408D91CEB88
:10047000030300F1FF382FD29E422DD90238634486
:100480009B1B89B2B3FBF7F607FB163341EA034126
:1004900006FB0EF38B4208D91CEB010106F1FF3875
:1004A00016D28B4214D9023E6144C91A46EA00466C
:1004B00038E72E46284605E70646E3E61846F8E6FE
:1004C0004B45A9D2B9EB020864EB0C0E0138A3E747
:1004D0004646EAE7204694E74046D1E7D0467BE728
:1004E000023B614432E7304609E76444023842E7A0
:1004F000704700BF02E000F000F8FEE772B6374830
:1005000080F30888364880F3098836483649086001
:1005100040F20000CCF200004EF63471CEF2000141
:100520000860BFF34F8FBFF36F8F40F20000C0F23F
:10053000F0004EF68851CEF200010860BFF34F8FF5
:10054000BFF36F8F4FF00000E1EE100A4EF63C71E2
:10055000CEF200010860062080F31488BFF36F8F8D
:1005600003F05CFE03F0EEFE4FF055301F491B4ACE
:1005700091423CBF41F8040BFAE71D49184A9142E9
:100580003CBF41F8040BFAE71A491B4A1B4B9A423D
:100590003EBF51F8040B42F8040BF8E7002018495D
:1005A000184A91423CBF41F8040BFAE703F03AFEC7
:1005B00003F00EFF144C154DAC4203DA54F8041B43
:1005C0008847F9E700F042F8114C124DAC4203DACB
:1005D00054F8041B8847F9E703F022BE0009002005
:1005E000001100200000000808ED00E000010020DC
:1005F00000090020104A0008001100207C11002092
:1006000080110020D83E0020E0010008E40100082D
:10061000E4010008E40100082DE9F04F2DED108AF7
:10062000C1F80CD0C3689D46BDEC108ABDE8F08FC0
:10063000002383F311882846A047002003F09AFA8C
:10064000FEE703F0FDF900DFFEE70000F8B500F07B
:1006500021FE03F085FD074603F0D6FD0546D0BB1D
:10066000294B9F4237D001339F4237D0274B27F089
:10067000FF029A4235D1F8B200F044FC2E4642F215
:10068000107400F045FC08B10024264601F0BAF8C9
:1006900058B3032000F03EF80024264635B11C4B29
:1006A0009F4203D003F0A8FD00242646002003F05B
:1006B00061FD0EB100F044F800F05CFC00F0ECFDD0
:1006C00002F0DAF80546B4B900F09CFC4FF47A70F9
:1006D00003F056FAF7E72E460024D2E70446012637
:1006E000CFE706464FF47A74CBE7002CD6D04FF410
:1006F0007A740126D2E702F0BFF8431BA342E3D984
:1007000000F01EF8DCE700BF010007B0000008B0F1
:10071000263A09B0084B187003280CD8DFE800F01F
:1007200008050208022000F013BE022000F008BEF7
:10073000024B00225A607047801100208411002073
:1007400038B501F05FF830B1254B03221A70254B04
:1007500000225A6038BD244B244A19680131F9D06F
:1007600004339342F9D1224C1F4DD4F80428AA42F5
:10077000F0D3204B9B6803F1006303F5D0439A420A
:10078000E8D203F00BFD03F01DFD002000F09EFDFC
:100790000220FFF7BFFF184B9A6D00229A65996FF0
:1007A0009A67996FD96DDA65D96FDA67D96F196E63
:1007B0001A66D3F88010C3F88020D3F8803072B660
:1007C0004FF0E0233021C3F8085DD4F80038D4F8A6
:1007D000042881F311889D4683F308881047B9E700
:1007E00080110020841100200068000820680008A3
:1007F000006000080011002000100240094A136840
:1008000049F2690099B21B0C00FB01331360064BDF
:10081000186844F2506182B2000C01FB02001860BB
:1008200080B27047141100201011002010B5002173
:100830001022044600F0A6FD034B03CB206061604C
:100840001868A06010BD00BF9075FF1F2DE9F04132
:10085000ADF5507D0DF13C086EAC40F275120746C7
:100860000D4610A80021C8F8001000F08BFD4FF4D1
:10087000C4720021204600F085FD01F0FDFF254BEC
:100880004FF47A72B0FBF2F0186093E8070002238D
:1008900084E807000DF5ED702382FFF7C7FF41F2F2
:1008A00004631D49238407A803F0ECFF1C2384F88C
:1008B00032310DF2EB226B440DF1340C1E4603CEA7
:1008C000664510605160334602F10802F6D1306887
:1008D000106041460122204600F0A0FD0023039352
:1008E000AB7E029305F11903019380B20123CDE998
:1008F00004800093E97E05A3D3E90023384602F083
:1009000079FB0DF5507DBDE8F08100BF9E6AC421E2
:10091000818A46EE8C110020944800082DE9F041B0
:100920002C4C237ADAB080460D465BBB27A92846BB
:1009300000F084FE0746002842D19DF89D60C82E35
:100940003ED801464FF4A662204600F01BFD4FF44E
:100950008073C4F8F8314FF40073C4F80C334FF4CB
:100960004073C4F8203432460DF19E0104F10900B1
:1009700000F0F6FC26449DF89C30777223720BB988
:10098000EB7E23728122002106AC27A800F0FAFC3E
:100990000122214627A800F08DFE00230393AB7EA1
:1009A000029305F1190380B201932823CDE9044095
:1009B0000093E97E05A3D3E90023404602F01AFB29
:1009C0005AB0BDE8F08100BFAFF3008026417272DB
:1009D000DF25D7B788360020F0B5254E4FF48A754D
:1009E00005FB0065F1B096F8D83085F8DC300024BE
:1009F000D822214685F8E8403AA800F0C3FC06F169
:100A0000090000F0B7FCD5F8E4308DF8F000C2B270
:100A100006AF06F109010DF1F100CDE93A3400F01D
:100A20009FFC394601223AA800F070FE80B2CDE961
:100A3000047008230127CDE9023706F1D80301939A
:100A400030230093317A0B4807A3D3E9002302F047
:100A5000D1FAA04206DD01F00FFFC5F8E0003846EC
:100A600071B0F0BD2046FBE778F6339F93CACD8D79
:100A700088360020A42100202DE9F0411D4D1E4E96
:100A80001E4F86B0284602F0E1FA034658B3002410
:100A9000CDE90344ADF81440027B8DF81420996829
:100AA0004068029403AA03C21B68DFF8548043F035
:100AB0000043029301F0E2FE821941F10003009429
:100AC00002A9384601F0BAF8A04205DD284602F036
:100AD000C1FA88F80040D5E798F80030072B05D810
:100AE000013388F8003006B0BDE8F081014802F01B
:100AF000B1FAF8E7A421002040420F00D8210020DD
:100B0000BD3B002070B50D4614461E4602F0CEF9DE
:100B100050B9022E10D1012C0ED112A3D3E900231B
:100B2000C5E90023012007E0282C10D005D8012CAE
:100B300009D0052C0FD0002070BD302CFBD10BA3A9
:100B4000D3E90023ECE70BA3D3E90023E8E70BA3E9
:100B5000D3E90023E4E70BA3D3E90023E0E700BFD8
:100B6000AFF30080401DA12026812A0B78F6339F29
:100B700093CACD8D9E6AC421818A46EE2641727247
:100B8000DF25D7B7F017304A39059E5638B50546E8
:100B90000E4C0021013500F0BBFBA4F82C55B4F835
:100BA0002C0500F09DFB78B1B4F82C0500F0A8FBF3
:100BB000014648B9B4F82C0500F0AAFBB4F82C356E
:100BC0000133A4F82C35EAE738BD00BF8836002091
:100BD00010B50A4B0A4A1A6003F5805393F848206F
:100BE0003AB95C6C2CB1204600F08AFE204603F036
:100BF000FFFDBDE81040034800F082BED821002070
:100C0000E4480008083200202DE9F04F8FB000AF13
:100C100005460C4602F04AF9002849D1237E022BF2
:100C20001BD1E38A012B18D101F026FE0646FFF7FF
:100C3000E5FD03464FF4C870DFF8C482B3FBF0F261
:100C400006F5167602FB103316FA83F3C8F8003067
:100C5000E37E33B9A34B00221A703C37BD46BDE892
:100C6000F08F07F12401204600F0A6FC0028F4D103
:100C700007F11400FFF7DAFD97F8264007F1140199
:100C8000224607F1270003F0CBFD0028E2D10F2C0C
:100C900008D8944B1C70D8F80030A3F51673C8F828
:100CA0000030DAE797F82410284602F0F7F8D4E786
:100CB000E38A282B2BD010D8012B23D0052BCCD1A5
:100CC000BFF34F8F8849894BCA6802F4E06213432F
:100CD000CB60BFF34F8F00BFFDE7302BBDD1844EFB
:100CE000E17E327A9142B8D1607E3146002291F89D
:100CF000DC50854200F0A5800132042A01F58A719A
:100D0000F5D1AAE721462846FFF7A0FDA5E7214631
:100D10002846FFF703FEA0E7B2F8EC507B6005F130
:100D200003094FEA99094FEA8902D11DC908A8EBC6
:100D3000C1039D46EB460021584600F023FB04F119
:100D4000EE012A463144584600F00AFB7B6813B98D
:100D5000012000F0BBFA96F8D20000F0C1FA044678
:100D600030B9307200F0DCFA204600F0AFFAB1E0A2
:100D7000D6F8D4203AB996F8D200B6F82C2582429B
:100D800001D8FFF703FFD6F8D4202A44944208D2B2
:100D900096F8D200B6F82C250130824201D8FFF730
:100DA000F5FE70685FFA89F2594600F0F3FA08B967
:100DB000C54679E0726896F8D2002A447260D6F887
:100DC000D42005EB0209C6F8D49000F089FA8145D9
:100DD00009D396F8D220D6F8D4000132001B86F849
:100DE000D220C6F8D400FF2D0FD80024347200F0B2
:100DF00097FA204600F06AFA00F004FD3D4B188196
:100E000008B9FFF79DFCC54627E7BB6896F8D900EF
:100E10000AFB0362FB68D2F8E41082F8E83001F5BF
:100E20008061C2F8E030C2F8E410FFF7D5FDFFF7AB
:100E300023FE96F8D920013202F0030286F8D92069
:100E4000B6E74FF48A7A0AFB02F505F1EA0131446C
:100E5000204600F087FCF86000287FF4FEAE3544A1
:100E6000012285F8E82001F007FDD5F8E020D6ED55
:100E7000007ADFED216A801A192838BF192040F660
:100E8000B832904228BF1046B8EE677A07EE900A53
:100E9000F8EEE77A67EEA67ADFED186AE7EE267AD3
:100EA000FCEEE77AC6ED007A96F8D930BB60BA68F6
:100EB00073680AFB02F4321992F8E81059B1D2F8BB
:100EC000E4108B42E8463FF427AF002182F8E81097
:100ED000C2F8E010C5467368064A9B0A01331381C5
:100EE000BBE600BF9D21002000ED00E00400FA05F4
:100EF000883600208C110020CDCCCC3D6666663F44
:100F0000A0210020014B1870704700BF98110020ED
:100F100038B54FF00054134B22689A4220D1124B3F
:100F2000627D12481A70237D03724FF48073C0F8FB
:100F3000F8314FF40073C0F80C3300254FF44073C0
:100F4000C0F820340A49C0F8E450C922093000F042
:100F500007FAE0222946204600F014FA012038BDA5
:100F60000020FCE79AAD44C5981100208836002087
:100F70001600002037B500F045FC194D19492881AD
:100F800002236B7100220123174801F07FF8002330
:100F90000193164B164900931648174B4FF4805295
:100FA00001F054FF154B197811B1124801F076FF8A
:100FB00001F062FC0446FFF721FC4FF4C873B0FB5C
:100FC000F3F202FB130304F5167010FA83F00C4BD6
:100FD000186003F019F908B10F232B8103B030BD5D
:100FE0008C11002040420F00D8210020050B000882
:100FF0009C110020A4210020090C00089811002059
:10100000A02100202DE9F04F2DED028B90A7D7E90C
:1010100000670FF24429D9E90089884C95B00DADDD
:101020009FED848BFFF728FDDFF834B200230C938B
:10103000ADF83C300D936B6000230DF125028DED72
:10104000008B4FF0010A09A958468DF825308DF81C
:1010500024A001F079FB9DF824200023002A40F011
:10106000AF80204601F022FF0546002847D1DFF877
:10107000F4B101F001FCDBF8003098423FD301F0FD
:10108000FBFB0790FFF7BAFB079A4FF4C873B0FB5E
:10109000F3F101FB130302F5167010FA83F0CBF89D
:1010A0000000DFF8C4B19BF800100791002914BFBD
:1010B0002B46534610A88DF83030FFF7B7FB079941
:1010C000C1F11002D2B2062A10AB28BF0622194481
:1010D0000DF13100079200F043F9079A0CAB03932E
:1010E000182302930132564BD2B2CDE900A30492E9
:1010F0003B463246204601F01FFF8BF8005001F0BE
:10110000BBFB504A504D1368C31AB3F57A7F32D3F4
:10111000106001F0B3FB02460B46204601F0A4FF2D
:10112000204601F0C3FE30B32B7ADFF840A1002B3C
:1011300014BF032302238AF8053001F09DFB0DF153
:10114000400B4FF47A730122B0FBF3F05946CAF812
:101150000000504600F008FA182302933B4B01931D
:1011600080B240F25513CDE903B0009342464B469E
:10117000204601F0E1FE2B7AB3B101F07DFB4FF088
:10118000000A83464FF48A7295F8D900504400F063
:10119000030002FB005393F8E810002934D00AF151
:1011A000010ABAF1040FEFD1C82002F0E9FC2B7A52
:1011B000002B7FF434AF15B0BDEC028BBDE8F08F8F
:1011C0004FF0904110A84A6982F040024A611946E6
:1011D000102200F0D7F80DF126030AAA0CA95846F0
:1011E00000F01EFE95E8030011AB83E803009DF8B4
:1011F0003C308DF84C300C9B109310A9DDE90A238C
:10120000204602F005F917E7D3F8E01049B12B6842
:10121000FA2B38BFFA23ABEB01010533B1EB430FD7
:10122000BDD3FFF7D9FB4FF48A720028B7D1BBE7D3
:10123000AFF300800000000000000000A4210020A7
:101240009C210020B83B002088360020BC3B0020B9
:10125000401DA12026812A0BF1C6A7C1D068080F26
:10126000D8210020A02100209D2100208C110020E9
:1012700008B5054800F078FEBDE80840034A044977
:10128000002003F0AFBA00BFD8210020F83B0020B7
:10129000D10B00087047000070B502F0FDFD094E4B
:1012A000094D3080002428683388834208D902F031
:1012B000EFFD2B6804440133B4F5D04F2B60F2D31B
:1012C00070BD00BFEC3B0020C03B002002F096BE8A
:1012D00000F10060920000F5D04002F019BE00005D
:1012E000054B1A68054B1B889B1A834202D9104490
:1012F00002F0CEBD00207047C03B0020EC3B002038
:10130000024B1B68184402F0C9BD00BFC03B00205F
:10131000024B1B68184402F0D3BD00BFC03B002045
:10132000064991F8243033B10023086A81F824304B
:101330000822FFF7CDBF0120704700BFC43B00204B
:10134000022802BF4FF0904340229A61704700008C
:10135000022802BF4FF090434FF480029A61704719
:1013600010B50023934203D0CC5CC4540133F9E799
:1013700010BD000003460246D01A12F9011B0029D5
:10138000FAD1704702440346934202D003F8011B8E
:10139000FAE770472DE9F8431F4D144695F82420CD
:1013A0000746884652BBDFF870909CB395F824300E
:1013B0002BB92022FF2148462F62FFF7E3FF95F863
:1013C0002400C0F10802A24228BF2246D6B24146FC
:1013D000920005EB8000FFF7C3FF95F82430A41BB3
:1013E0001E44F6B2082E17449044E4B285F82460F7
:1013F000DBD1FFF795FF0028D7D108E02B6A03EB7C
:1014000082038342CFD0FFF78BFF0028CBD100208F
:10141000BDE8F8830120FBE7C43B00202DE9F0473D
:101420000D46044600219046284640F27912FFF707
:10143000A9FF234620220021284601F08BFF231D0F
:1014400002222021284601F085FF631D032222216C
:10145000284601F07FFFA31D03222521284601F025
:1014600079FF04F1080310222821284601F072FFB9
:1014700004F1100308223821284601F06BFF04F123
:10148000110308224021284601F064FF04F11203F1
:1014900008224821284601F05DFF04F114032022B0
:1014A0005021284601F056FF04F118034022702114
:1014B000284601F04FFF04F120030822B0212846FE
:1014C00001F048FF04F121030822B821284601F069
:1014D00041FF04F12207C0263B4631460822284638
:1014E000083601F037FFB6F5A07F07F10107F3D109
:1014F00004F1320308223146284601F02BFF002771
:1015000004F1330A94F832304FEAC7099F4209F5D3
:10151000A47615D3B8F1000F08D1314604F59973BC
:101520000722284601F016FF09F24F16274694F8C5
:1015300032213B1B93420CD3F01DC008BDE8F0875D
:101540000AEB070308223146284601F003FF013762
:10155000D8E707F2331331460822284601F0FAFE95
:1015600008360137E3E7000013B5044608460021BA
:1015700001602346C0F803102022019001F0EAFE2A
:101580000198231D0222202101F0E4FE0198631D31
:101590000322222101F0DEFE0198A31D0322252152
:1015A00001F0D8FE019804F108031022282101F06F
:1015B000D1FE072002B010BDF7B50023047F0091D3
:1015C0000E4607221946054601F088FD731C00935C
:1015D000012200230721284601F080FDC4B9B31C75
:1015E0000093052223460821284601F077FD0D24AB
:1015F0003746B278BB1B934211D32B7FA88A07349E
:10160000E408BBB9844294BF0020012003B0F0BDC0
:10161000AB8ADB00083BDB08B3700824E8E7FB1C5F
:101620000093214600230822284601F057FD083484
:101630000137DEE7201A18BF0120E7E7F7B50023DE
:10164000047F00910E4608221946054601F046FD2A
:10165000731CC4B90822009311462346284601F0A2
:101660003DFD1024012372785F1C013B934211D38E
:101670002B7FA88A0734E408BBB9844294BF0020BA
:10168000012003B0F0BDAB8ADB00083BDB087370C0
:101690000824E7E7F319009321460023082228468F
:1016A00001F01CFD08343B46DDE7201A18BF01207D
:1016B000E7E70000F8B50E460546144600218122F2
:1016C0003046FFF75FFE2B4608220021304601F02E
:1016D00041FE7CB96B1C07220821304601F03AFE1E
:1016E0000F2401236A785F1C013B934204D3E01D61
:1016F000C008F8BD0824F4E7EB192146082230465B
:1017000001F028FE08343B46ECE70000F8B50E4631
:10171000054614460021CE223046FFF733FE2B4605
:1017200028220021304601F015FE7CB905F108039E
:1017300008222821304601F00DFE30242F462A7A57
:101740007B1B934204D3E01DC008F8BD2824F5E7B5
:1017500007F1090321460822304601F0FBFD083459
:101760000137ECE7F7B5047F00910E460123102204
:101770000021054601F0B2FCC4B9B31C0093092254
:1017800023461021284601F0A9FC19243746728807
:10179000BB1B9A4211D82B7FA88A0734E408BBB937
:1017A000844294BF0020012003B0F0BDAB8ADB006F
:1017B000103BDB0873801024E8E73B1D00932146B3
:1017C00000230822284601F089FC08340137DEE7AF
:1017D000201A18BF0120E7E730B5094D0A449142AD
:1017E0000DD011F8013B5840082340F30004013BA1
:1017F0002C4013F0FF0384EA5000F6D1EFE730BD30
:101800002083B8EDF7B5384A106851686B4603C3BA
:101810006A4636493648082303F012F80446002881
:1018200033D10A25334A106851686B4603C36A46B0
:1018300031492F48082303F003F80446002849D013
:101840000369B3F5CC3F45D8B0F8661040F21642B4
:1018500091423FD1294A024402F15C018B4239D3C3
:101860005C3B234900209E1AFFF7B6FF324607462D
:1018700004F164010020FFF7AFFFA3689F4229D164
:10188000E368984208BF002524E00369B3F5CC3F24
:1018900027D8418B40F21642914220D1174A024488
:1018A00002F110018B4218D3103B114900209D1A00
:1018B000FFF792FF2A46064604F118010020FFF7C1
:1018C0008BFFA3689E4202D1E368984201D00D25A8
:1018D000A8E70025284603B0F0BD1025A2E70C2597
:1018E000A0E70B259EE700BFB4480008DC97010085
:1018F00000680008BD480008909701000898FFF7AD
:1019000010B5037C044613B9006802F081FF20463D
:1019100010BD00000023BFF35B8FC360BFF35B8F7C
:10192000BFF35B8F8360BFF35B8F7047BFF35B8F49
:101930000068BFF35B8F704770B505460C30FFF74A
:10194000F5FF05F1080604463046FFF7EFFFA04219
:1019500006D930466D68FFF7E9FF2544281A70BDA7
:101960003046FFF7E3FF201AF9E7000070B505469F
:10197000406898B105F10800FFF7D8FF05F10C06A3
:1019800004463046FFF7D2FF8442304694BF6D686C
:101990000025FFF7CBFF013C2C44201A70BD00004E
:1019A00038B50C460546FFF7C7FFA04210D305F136
:1019B0000800FFF7BBFF04446868B4FBF0F100FBCC
:1019C0001144BFF35B8F0120AC60BFF35B8F38BD68
:1019D0000020FCE72DE9F041144607460D46FFF7CD
:1019E000C5FF844228BF0446D4B1B84658F80C6BF2
:1019F0004046FFF79BFF3044286040467E68FFF773
:101A000095FF331A9C4203D86C600120BDE8F08139
:101A10006B60A41B3B68AB602044E8600220F5E7E4
:101A20002046F3E738B50C460546FFF79FFFA04276
:101A300010D305F10C00FFF779FF04446868B4FB8C
:101A4000F0F100FB1144BFF35B8F0120EC60BFF3AA
:101A50005B8F38BD0020FCE72DE9FF4188466946D1
:101A60000746FFF7B7FF6C4606B204EBC606002533
:101A7000B44209D06268206808EB0501FFF770FCEA
:101A8000636808341D44F3E729463846FFF7CAFF68
:101A9000284604B0BDE8F081F8B505460C300F4685
:101AA000FFF744FF05F1080604463046FFF73EFF06
:101AB000A042304688BF6C68FFF738FF201A3860B4
:101AC00020B130462C68FFF731FF2044F8BD0000FC
:101AD00073B5144606460D46FFF72EFF844228BF15
:101AE00004460190DCB101A93046FFF7D5FF019B08
:101AF00033B93268C5E90233C5E9002401200CE09E
:101B00009C4238BF01942860019868608442F5D9EE
:101B10003368AB60241AEC60022002B070BD20462E
:101B2000FBE700002DE9FF410F466946FFF7D0FFB4
:101B30006C4600B204EBC0050026AC4209D0D4F8D4
:101B4000048054F8081BB8194246FFF709FC4644C4
:101B5000F3E7304604B0BDE8F081000038B5054633
:101B6000FFF7E0FF044601462846FFF719FF20462D
:101B700038BD0000302383F3118862B6704700003F
:101B8000002383F3118862B670470000012070477C
:101B90007047000010B41346026814680022A4467F
:101BA0005DF8044B6047000000F5805090F8590440
:101BB0007047000000F5805090F852047047000014
:101BC00000F5805090F9580470470000502070478D
:101BD00000F5805208B5FFF7CDFFD2F89834D2F85F
:101BE00094041844D2F890341844D2F87834184445
:101BF000D2F888341844D2F884341844FFF7C0FF70
:101C000008BD000038B5C26A936923F001039361EF
:101C1000044600F031FE0546E36A9B69DB0706D502
:101C200000F02AFE431BFA2BF6D9002004E004F54D
:101C30008054012084F8520438BD00002DE9F04F93
:101C40000C4600F5805185B01F4691F85234BDF81E
:101C50003890054690469BB1D1F874340133C1F8F1
:101C6000743423689A0006D4237B082B0BD9627B3B
:101C70000AB10F2B07D9D1F878340133C1F8783481
:101C80004FF0FF300FE0FFF775FFEB6AD3F8C42089
:101C900012F4001A0AD0D1F87C340133C1F87C3434
:101CA000FFF76EFF002005B0BDE8F08FD3F8C460E9
:101CB00022686B6AC6F301464FF0480B002A1BFBF3
:101CC000063BB4BF42F080429204CBF80020236868
:101CD0005B0044BF42F00052CBF80020227B330669
:101CE00043EA0243CBF80430607B720118B343F43B
:101CF0004013CBF80430D1F8A4340133C1F8A43434
:101D0000AB1803F58353197B41F020011973207B35
:101D1000039200F00DFE039A033080105FFA8AF3FD
:101D200083420AF1010A0DDA04EB83010BEB830312
:101D300049689960F2E7AB1803F58353197B60F3A8
:101D40004511E3E7EB6A0121B140C3F8CC10AB18B1
:101D500003F58253C3E9048705EB461303F5825369
:101D60002146183304F10C0051F804CB43F804CB9E
:101D70008142F9D1098819802A4441F26803284632
:101D8000D65002F5805209F0030392F86C1043F02C
:101D9000100321F01F010B4382F86C30FFF7F0FEB7
:101DA0004246CDF800903B46214600F087FD0120D9
:101DB00079E7000013B500F580540191606CFFF7DE
:101DC000D5FD1F280AD90199606C2022FFF744FE37
:101DD000A0F120035842584102B010BD0020FBE79B
:101DE00008B500F58050FFF7C5FE406CFFF792FD87
:101DF000BDE80840FFF7C4BE002202608281426055
:101E00008260704710B500220023C0E90023002340
:101E1000044603810C30FFF7EFFF204610BD0000A1
:101E20002DE9F047074688B007F5805468469A4682
:101E30008846FFF79FFE9146FFF7E4FF606CFFF7CF
:101E40007BFD1F282CD9606C20226946FFF786FE97
:101E5000202825D194F8523413B303AD444605AB82
:101E60002E4603CE9E4220606160354604F1080490
:101E7000F6D130682060B388A380DDE90023C9E98A
:101E80000023BDF80830AAF80030FFF779FE4A4673
:101E900053464146384608B0BDE8F04700F0FCBC68
:101EA000FFF76EFE002008B0BDE8F0872DE9F84F7F
:101EB00000230646C0E90133284B46F8303B00F5C5
:101EC0008154054688463746103438462037FFF798
:101ED00099FFA742F9D105F580544FF4805326634A
:101EE0000026C4E90D366764012305F5835705F51F
:101EF000A359E66384F8403084F84830103709F17C
:101F000010094FF0000A4FF0000B47E908ABA7F1AA
:101F10001800FFF771FF203747F8286C4F45F4D1C0
:101F200084F85884A4F85A64A4F85C64A4F85E6445
:101F300084F86064A4F86264A4F86464A4F8666435
:101F400084F86864B8F1000F02D0054800F08EFCF8
:101F5000044BEB622846BDE8F88F00BFE448000858
:101F6000C84800080064004010B5044B19780446C6
:101F70004A1C1A70FFF79AFF204610BDF53B00205F
:101F80002DE9F04300295FD03048314BB3FBF1F32A
:101F900081428CBF0A201120451EB3FBF0F700FBE5
:101FA0001730ECB220B1022D2846F5D8002037E0DA
:101FB0007D1EB5F5806F33D2C4EBC40808F103036E
:101FC0004FEAE30EC3F3C703A4EB030C0EF10109C0
:101FD0004FF47A705FFA8CF60EFB000E59FA8CFC07
:101FE000BEFBFCFCBCF5617F1CDC1FFA8CF4581CAA
:101FF00056FA80F047431648B0FBF7F7B942D5D1FF
:10200000013BDBB20F2BD1D8711EC9B207294FF0AB
:10201000000005D810711480558053719171012012
:10202000BDE8F08308F1FF334FEAE30CC3F3C703C5
:10203000E41A0CF1010EE6B20CFB00005EFA84F427
:10204000B0FBF4F4A4B2D2E70846E9E73F420F0040
:1020500000366E010B4B10B54FF45472044600214C
:102060001846FFF78FF9084BA3614033E361D8337B
:102070002362F0336362E36A60610022C3F8C02028
:1020800010BD00BF00A4004070A400402DE9F04F37
:1020900000F58055994695F85834012B89B00446CF
:1020A0008A46904604D90027384609B0BDE8F08F2B
:1020B0008D4A52F8231009B942F823008B49C4F81D
:1020C0000CA00B7884F8109093B9FFF753FD884B60
:1020D0009A6D42F000729A659A6B42F000729A63B0
:1020E0009A6B22F000729A6301230B70FFF748FD90
:1020F00095F8513473B903211520FFF73BFD01F02A
:1021000015FC0321162001F011FC012385F8513440
:10211000FFF736FDFFF72EFDE26A936923F0100307
:10212000936100F0A9FB0746E36A9E6916F0080672
:1021300007D000F0A1FBC31BFA2BF5D9FFF720FD58
:10214000B1E79A6942F001029A6100F095FB0746F7
:10215000E36A9A69D00705D400F08EFBC31BFA2B03
:10216000F6D9EBE79A6942F002029A61E36A002726
:102170005F65FFF705FD686CFFF7CCFB04F5825B3C
:102180000BF1100B202200216846FFF7FBF802A894
:10219000FFF732FE06976A460BEB06030DF1180EA9
:1021A0009446BCE80300F44518605960624603F1A8
:1021B0000803F5D1DCF80000186020369CF80420F4
:1021C0001A71B6F5806FDDD1002304F5A25285F8AF
:1021D000503485F853341A3251462046FFF7D0FE6A
:1021E000074690B9E26A936923F00103936100F016
:1021F00043FB0546E36A9B69D9077FF554AF00F0BE
:102200003BFB431BFA2BF5D94DE795F85F6495F836
:102210005E24C5F86CA4360246EA426695F860244E
:10222000E36A1643B5F85C2446EA0246DE61B8F17B
:10223000000F29D004F5A352023241462046FFF791
:102240009FFE90B9E26A936923F00103936100F065
:1022500013FB0546E36A9B69DA077FF524AF00F0BC
:102260000BFB431BFA2BF5D91DE795F8683495F85D
:102270006714C5F870841B0143EA0123B5F86414A0
:10228000E26A43EA0143D3602046FFF7E3FE0023FE
:1022900085F85934E36A6FF040421A65E36A154ADB
:1022A0005A65E36A44229A65E36A0722C3F8DC2090
:1022B000E36A03229145DA653FF4F6AEE26A936978
:1022C00023F00103936100F0D7FA0646E36A9B69A5
:1022D000DB0705D500F0D0FA831BFA2BF6D9E2E62E
:1022E000012385F85234DFE6F03B0020F43B002068
:1022F000001002409B0008002DE9F04F054689B010
:1023000090469946002741F2680A00F58056EB6A2C
:10231000D3F8D430FB40D8074AD505EB47125244D6
:102320004FEA471B1379190742D4D6F8803401339A
:10233000C6F8803413799A0648BFD6F8A83405EB5E
:102340000B0248BF0133524448BFC6F8A834137982
:1023500043F008031371DB0722D596F85334FBB121
:1023600005F58254183468465C44FFF74BFD03AB17
:1023700004F1080C206861681A4603C208346445F9
:102380001346F7D120681060A2889A800123ADF827
:1023900008302B68CDE90089DB6B694628469847F1
:1023A000D6F8543423B1D6F89C340133C6F89C34A3
:1023B0000137202FABD109B0BDE8F08F2DE9F04FE8
:1023C0008DB004460F4600F059FA82468946002F28
:1023D00056D1E36AD3F89020920141BF04F58051B1
:1023E000D1F894240132C1F89424D3F89020160730
:1023F00003D100200DB0BDE8F08FD3F89050E6690E
:10240000C5F30125482303FB0566E8464046FFF770
:10241000F3FC326851004ABF22F06043C2F38A43A2
:1024200043F00043920048BF43F080430093736839
:1024300013F400131FBF04F5805201238DF80D30F3
:10244000D2F8AC340EBF8DF80D300133C2F8AC3485
:10245000F38803F00F038DF80C304FF0000B9DF85C
:102460000C0000F065FA5FFA8BF3984220D9F2185D
:102470000CA90B44127A03F82C2C0BF1010BEEE79C
:10248000012FB6D1E36AD3F89820950141BF04F536
:102490008051D1F894240132C1F89424D3F89820C3
:1024A0001007A6D0D3F89850266AC5F30125A9E7EE
:1024B000EFB9E36AC3F8945004A8FFF7A3FC98E8C7
:1024C0000F0007AD07C52B800023ADF81830236837
:1024D0002046CDE904A9DB6B04A9984704F5805494
:1024E00058B1D4F88C340133C4F88C3482E7012F0E
:1024F00004BFE36AC3F89C50DEE7D4F8903401339C
:10250000C4F89034012075E7F8B505460F4600F58C
:102510008054012639462846FFF750FF10B184F851
:102520005364F7E7D4F8543423B1D4F89C3401331E
:10253000C4F89C34F8BD0000F0B5C36A1A6C12F4FC
:102540007F0F2BD000F580541B6CC4F8A03441F2EF
:102550006805002347194FF0010C00EB43122A4491
:102560005E01117911F0020F15D0490713D4B95942
:10257000C66AD6F8C8E00CFA01F111EA0E0F0AD0CB
:10258000C6F8D010117941F004011171D4F88824F3
:102590000132C4F888240133202BDED1F0BD0000C5
:1025A00010B5254C254B226802B338B31A6D1206BC
:1025B0000ED580221A6500F061F950EA01020B463F
:1025C00002D0013861F1000302462068FFF794FE53
:1025D0001A4A136D1B032AD523684FF4002103F513
:1025E00080531165012283F8592420E001221A65E5
:1025F00008221A654FF480621A6510BD196DC8076C
:1026000002D4196D890705D50321196510460021EB
:10261000FFF77AFF094B1A6D100702D41A6DD10625
:1026200005D518221A6520680121FFF76DFF206883
:10263000BDE81040FFF780BFF03B00200064004081
:1026400008B5FFF797FAFFF777FFBDE80840FFF7F7
:1026500097BA0000C36AD3F8C40080F40010C0F336
:102660004050704700F5805008B5FFF783FA406C82
:10267000FFF762F9FFF784FA43090CBF012000203D
:1026800008BD000000F5805393F8592462B1C16A77
:102690008A6922F001028A61D3F898240132C3F8D2
:1026A0009824002283F85924704700002DE9F7434D
:1026B00000F5825198461031FFF75CFA002541F28F
:1026C000680E4FF0010900F5805C00EB451474447E
:1026D00023795E071CD4DB061AD5C36A8E69D3F84A
:1026E000C87009FA06F63E4212D04F6801970F688B
:1026F0009742019F77EB08070AD2C3F8D06023798D
:1027000043F004032371DCF884340133CCF88434BF
:102710000135202D01F12001D7D103B0BDE8F043F0
:10272000FFF72EBAF8B51E46002313700F46054674
:102730001446FFF797FF80F0010038701EB128465D
:10274000FFF788FF2070F8BD2DE9F04F85B099465E
:10275000DDE90EA30D4602931378019391F800B0C2
:102760008046164600F08AF82B7804460F4613B9C7
:102770003378002B42D022463B464046FFF796FF77
:10278000FFF75EFFFFF77EFF4B4632462946FFF715
:10279000C9FF2B7833B1BBF1000F03D0012005B086
:1027A000BDE8F08F337813B1019B002BF6D108F50B
:1027B00080530393029B544577EB03031ED2039B84
:1027C000D3F85404D0B10368AAEB0401DB6889B2E2
:1027D00098474B46324629464046FFF7A3FF2B78E1
:1027E00013B1BBF1000FD9D1337813B1019B002B8A
:1027F000D4D100F043F804460F46DBE70020CEE7D3
:1028000008B50020FFF7CCFEBDE8084001F050B845
:1028100008B50120FFF7C4FEBDE8084001F048B844
:1028200000B59BB0EFF3098168226846FEF798FD7A
:10283000EFF30583014B9B6BFEE700BF00ED00E06B
:1028400008B5FFF7EDFF000000B59BB0EFF309817D
:1028500068226846FEF784FDEFF30583014B5B6B4E
:10286000FEE700BF00ED00E0FEE700000FB408B592
:10287000029801F01BF9FEE701F00EBC01F0E6BB87
:1028800013B56C4684E80600031D94E8030083E852
:102890000500012002B010BD73B58568019155B1E6
:1028A0001B885B0707D4D0E900369B6B9847019AD9
:1028B000C1B23046A847012002B070BDF0B58668AD
:1028C00089B005460C465EB1BDF838305B070AD4C6
:1028D000D0E900379B6B98472246C1B23846B047D3
:1028E000012009B0F0BD00220023CDE90023002320
:1028F000ADF808300A4603AB01F1080610685168CC
:102900001C4603C40832B2422346F7D11068206047
:102910009288A280FFF7B2FF0423ADF808302B683D
:10292000CDE90001DB6B694628469847D8E70000EF
:10293000082817D909280CD00A280CD00B280CD04D
:102940000C280CD00D280CD00E2814BF40203020AD
:1029500070470C20704710207047142070471820D3
:1029600070472020704700002DE9F041456A15B9F5
:102970004162BDE8F0814B6823F06047C3F38A46AB
:102980004FEAD37EC3F3807816EA230638BF3E466B
:10299000AC462B465A68BEEBD27F22F060440AD088
:1029A000002A18DAA40CB44217D19D420FD10D6051
:1029B000DEE71346EEE7A74207D102F08044C2F3F8
:1029C000807242450BD054B1EFE708D2EDE7CCF866
:1029D00000100B60CDE7B44201D0B442E5D81A68CC
:1029E0009C46002AE5D11960C3E700002DE9F047B5
:1029F000089D01F007044FEAD508224405F00705B9
:102A000000EBD1004FF47F49944201D1BDE8F0873B
:102A100004F0070705F0070A57453E4638BF5646FB
:102A2000C6F10806111B8E4228BF0E46E10808EBCE
:102A3000D50E415C13F80EC0B94029FA06F721FA09
:102A40000AF1FFB28CEA010147FA0AF739408CEA31
:102A5000010C03F80EC034443544D5E780EA012068
:102A6000082341F2210201B24000002980B203F1A3
:102A7000FF33B8BF504013F0FF03F4D1704700009C
:102A800038B50C468D18A54200D138BD14F8011B8D
:102A9000FFF7E4FFF7E7000042684AB113684360BC
:102AA0004389818901339BB29942438138BF838135
:102AB0001046704770B588B0202204460D4668461F
:102AC0000021FEF75FFC20460495FFF7E5FF024674
:102AD00058B16B46054608AE1C4603CCB44228608C
:102AE0006960234605F10805F6D1104608B070BDAF
:102AF000082817D909280CD00A280CD00B280CD08C
:102B00000C280CD00D280CD00E2814BF40203020EB
:102B100070470C2070471020704714207047182011
:102B20007047202070470000082817D90C280CD9BE
:102B300010280CD914280CD918280CD920280CD905
:102B400030288CBF0F200E207047092070470A20C4
:102B500070470B2070470C2070470D207047000015
:102B60002DE9F843078C072F04461ED9D0E90298B7
:102B700000254FF6FF73C5F12006A5F1200029FAC4
:102B800005F108FA06F628FA00F031430143C9B20C
:102B90001846FFF763FF0835402D0346EBD1E16986
:102BA0003A46BDE8F843FFF76BBF4FF6FF70BDE84C
:102BB000F883000010B54B6823B9CA8A63F3090291
:102BC000CA8210BD04691A681C600361C38A013B94
:102BD000C3824A60EFE700002DE9F84F1D46CB8A1B
:102BE0000F46C3F309010529814692460B4630D0B2
:102BF0000020AAB207F11A049EB2042E1FFA80F830
:102C00000FD8904503F1010306D3FB8A0A4462F30F
:102C10000903FB8201201AE01AF80060E654013033
:102C2000EAE79045F1D2A1F1050B1C237C68BBFBC0
:102C3000F3F203FB12BB1FFA8BF6002C45D148467A
:102C4000FFF72AFF044638B978606FF00200BDE84C
:102C5000F88F4FF00008E6E7002606607860ADB216
:102C60004FF0000B454510D90AEB0803221D13F85D
:102C7000011B9155B1B208F101081B291FFA88F810
:102C80002BD0454506F10106F1D8FB8AC3F30902B2
:102C9000154465F30903BCE7013292B21C46236870
:102CA000002BF9D16B1F0B441C21B3FBF1F3013353
:102CB0009BB29A42D3D2BBF1000FD0D14846FFF766
:102CC000EBFE20B9C4F800B0BFE70122E7E7C0F887
:102CD00000B05E4620600446C1E74545D5D9484668
:102CE000FFF7DAFE08B92060AFE7C0F800B00026B1
:102CF00020600446B6E700002DE9F04F2DED028B71
:102D00001C4683B05B69019207468846002B00F0A1
:102D10009A80238C2BB1E269002A00F09480072B63
:102D200035D807F10C00FFF7B7FE054638B96FF04C
:102D30000205284603B0BDEC028BBDE8F08F1422DB
:102D40000021FEF71FFB228CE16905F10800FEF768
:102D500007FB208C013080B2FFF7E6FEFFF7C8FECC
:102D6000013880B22084013028746369228C1B787A
:102D70002A4403F01F0363F03F0348F0004113723D
:102D8000384669602946FFF7EFFD0125D1E700F1DC
:102D90000C034FF0000908EE103A4FF0800A4E463F
:102DA0004D4618EE100AFFF777FE83460028BED086
:102DB00014220021FEF7E6FA002E3AD1019BABF86F
:102DC000083002220BF1080E1FFA82FC0CF1010000
:102DD000BCF1060F218C80B201D88E422BD3FFF7B5
:102DE000A3FEFFF785FE62691278013802F01F0228
:102DF0008E4208BF4FF0400A42EA49121BFA80F1A6
:102E00004AEA020A013048F0004281F808A08BF833
:102E10001000CBF8042059463846FFF7A5FD238C57
:102E20000135B3422DB289F001094FF0000AB8D143
:102E30007FE70022C6E7E169895D0EF802100136DE
:102E4000B6B20132C0E76FF0010572E7F8B515467A
:102E50000E463022002104461F46FEF793FA069BD9
:102E60006360B5F5001F079BA76034BF6A094FF682
:102E7000FF72A36297B2E66104F1100000239A4248
:102E800006D800230360A782E3822383E360F8BDB2
:102E90000660013330462036F1E7000003781BB9A5
:102EA0004BB2002BC8BF017070470000007870471C
:102EB000F8B50C46C969074611B9238C002B37D1E8
:102EC000257E1F2D34D8387828BB228C072A2CD891
:102ED000268A36F003032BD14FF6FF70FFF7D0FDA3
:102EE00020F001003102400441EA0561400C41EA52
:102EF00040254FF6FF72234629463846FFF7FCFE71
:102F0000002807DD626913780133DBB21F2B88BF0D
:102F100000231370F8BD218A2D0645EA01250543DB
:102F20002046FFF71DFE0246E5E76FF00300F1E7DC
:102F30006FF00100EEE7000070B58AB00446164657
:102F40000021282268461D46FEF71CFABDF83830DD
:102F5000ADF810300F9B05939DF840308DF8183078
:102F6000119B07936946BDF84830ADF820302046E4
:102F7000CDE90265FFF79CFF0AB070BD2DE9F04175
:102F8000D36905460C4616460BB9138C5BBB377EDE
:102F90001F2F28D895F80080B8F1000F26D03046B2
:102FA000FFF7DEFD3378210241EAC33141EA08012F
:102FB000338A41EA076141EA03410246334641F060
:102FC00080012846FFF798FE00280ADD3378012BA0
:102FD00007D1726913780133DBB21F2B88BF00233E
:102FE0001370BDE8F0816FF00100FAE76FF00300A5
:102FF000F7E70000F0B58BB004460D4617460021F8
:10300000282268461E46FEF7BDF99DF84C305A1E30
:10301000534253418DF800309DF84030ADF81030E8
:10302000119B05939DF848308DF81830149B079339
:103030006A46BDF85430ADF8203029462046CDE927
:103040000276FFF79BFF0BB0F0BD0000406A00B1B5
:1030500004307047436A1A68426202691A60036169
:10306000C38A013BC38270472DE9F041D0F820802C
:10307000194E14461D464146002709B9BDE8F081A6
:10308000D1E90223A21A65EB0303964277EB03030F
:103090001ED2036A8B420DD1FFF78CFD036A1B68B9
:1030A000036203690B60C38A0161016A013BC38249
:1030B0008846E2E7FFF77EFD0B68C8F80030036939
:1030C0000B60C38A0161013BC382D8F80010D4E7CA
:1030D00088460968D1E700BF80841E002DE9F04FC3
:1030E0008BB00D46DDF8509014469B468046002874
:1030F00000F01981B9F1000F00F01581531E3F2B2C
:1031000000F21181012A03D1BBF1000F40F00B81C5
:103110000023CDE90833B8F81430B5EBC30F4FEAFC
:10312000C30703D300200BB0BDE8F08F2B199F42DB
:10313000D8F80C303ABF7F1BFFB227461BB9D8F82E
:103140001030002B7AD0272D4ED8C5F12806B74273
:103150004FF000032CBFF6B23E4600932946D8F844
:10316000080008AB3246FFF741FCA7EB060A3544DE
:103170005FFA8AFAB8F8143003F10053053BDB001C
:103180000493D8F80C3003932821039B13B1BAF1B0
:10319000000F2CD1D8F8100040B1BAF1000F05D0C3
:1031A000009608AB5246691AFFF720FC38B2002F90
:1031B000B8D066070AD00AAB03EBD401624211F81B
:1031C000083C02F00702134101F8083C082C3CD9E6
:1031D000102C40F2B580202C40F2B780BBF1000FDC
:1031E00000F09C80082334E0BA460026C2E7049B26
:1031F000E02B28BFE02306930B44AB42059314D980
:103200005A1B03980096924534BF5246D2B2691AAF
:1032100008AB04300792FFF7E9FB079A1644AAEBC4
:10322000020A1544F6B25FFA8AFA049B069A0599D7
:103230009B1A0493039B1B680393A6E70093D8F89B
:10324000080008AB3A462946AEE7BBF1000F13D0A1
:103250000123B4EBC30F6CD0082C12D89DF820309A
:10326000621E23FA02F2D50706D54FF0FF3202FAAA
:1032700004F423438DF820309DF8203089F8003085
:1032800051E7102C12D8BDF82030621E23FA02F24A
:10329000D10706D54FF0FF3202FA04F42343ADF80C
:1032A0002030BDF82030A9F800303CE7202C0FD8A2
:1032B0000899631E21FA03F3DA0705D54FF0FF32B0
:1032C00002FA04F40C430894089BC9F800302AE77A
:1032D000402C2BD0DDE90865611EC4F12102A4F168
:1032E000210326FA01F105FA02F225FA03F311434C
:1032F0001943CB0712D50122A4F12003C4F1200108
:1033000002FA03F322FA01F1A240524243EA010316
:1033100063EB430332432B43CDE90823DDE9082364
:10332000C9E90023FFE66FF00100FCE66FF008003A
:10333000F9E6082CA0D9102CB3D9202CEED8C3E77D
:10334000BBF1000FADD0022383E7BBF1000FBBD070
:1033500004237EE730B5012A144638BF0124402CEF
:1033600085B028BF40240025012ACDE9025518D890
:103370001B788DF8083063070AD004AB03EBD40543
:10338000624215F8083C02F00702934005F8083C39
:10339000009103462246002102A8FFF727FB05B053
:1033A00030BD082AE4D9102A03D81B88ADF80830AC
:1033B000E1E7202A8DBFD3E900231B680293CDE902
:1033C0000223D8E710B5CB681BB98B600B618B82E9
:1033D00010BD04691A681C600361C38A013BC38283
:1033E000CA60F0E703064CBFC0F3C030022070474C
:1033F00008B50246FFF7F6FF022806D15306C2F3CE
:103400000F2001D100F0030008BDC2F30740FBE725
:103410002DE9F04F93B0CDE903230A680446104626
:10342000FFF7E0FF022814BFC2F306260026002A99
:103430000D46824680F2F28112F0C04940F0EE81E2
:10344000097B002900F0EA81022803D02378B342E7
:1034500040F0E781C2F304630693104602F07F0355
:103460000593FFF7C5FF059B29444FEA834848EAC7
:103470000A4848EA4668CE7800230022CDE90823AE
:10348000F309834648EA0008029367D0059B00933E
:1034900002466768534608A92046B847002800F04E
:1034A000C381276A4FB9414604F10C00FFF702FBC4
:1034B000074690B96FF0020054E03B6998450DD083
:1034C0003F68002FF9D1414604F10C00FFF7F2FAF2
:1034D00007460028EED0236A3B60276297F817C0A2
:1034E00006F01F08CCF3840CACEB08001FFA80FE3A
:1034F0000028B8BF0EF12000A8EB0C031FFA83FED2
:10350000D7E90221B8BF00B2002B0793BEBF0EF16E
:1035100020031BB2079352EA010338D0039BDFF864
:1035200024E39A1A049B4FF0000C63EB01019645CB
:103530007CEB01032BD36B7B97F81AE0734519D111
:10354000029B002B78D0012821DC7868F8B9DFF8DD
:10355000F0C2944570EB010316D337E0276A27B910
:103560006FF00C0013B0BDE8F08F3B699845B5D003
:103570003F68F4E7B24890427CEB010301D300209E
:10358000F0E7029B002BFAD0079B0F2B17DCFA7D8C
:10359000B30002F0030203F07C031343FB753946CA
:1035A0002046FFF707FB6B7BBB76029B3BB9FB7D9D
:1035B000C3F38402013262F38603FB75D0E76A7BB2
:1035C000BB7E9A42DBD1029B002B35D0B309022B84
:1035D00032D0039BBB60049BFB60142200210DA82A
:1035E000FDF7D0FE039B0A93049B0B932B1D0C93BA
:1035F0002B7BADF83EB0013BDBB2ADF83C30069B17
:103600008DF84230059B8DF8433094F82C308DF8BE
:1036100040A083F001038DF844308DF84180A36809
:103620000AA920469847FB7DC3F38403013303F0C6
:103630001F039B02FB82A2E7FB7DC6F34012B2EBA5
:10364000D31F40F0F480C3F38403434540F0F2807D
:10365000029A2B7BB609002A4DD0F2075DD4032BCA
:1036600040F2EB80039BBB60049BFB602B7BAE1D99
:10367000033BDBB23246394604F10C00FFF7ACFAEB
:1036800000280CDA39462046FFF794FAFB7DC3F395
:103690008403013303F01F039B02FB820AE7DDE989
:1036A0000884AB883B834FF6FF73C9F12000A9F172
:1036B000200228FA09F104FA00F0014324FA02F288
:1036C00011431846C9B2FFF7C9F909F10809B9F160
:1036D000400F0346E9D1B8822A7B033AD2B2314681
:1036E000FFF7CEF9FB7DB882DA43C2F3C01262F372
:1036F000C713FB7543E786B92E1D013BDBB232468B
:10370000394604F10C00FFF767FA0028BADB2A7B80
:10371000B88A013AD2B23146E2E7F98AC1F3090127
:10372000013B0429DAB25BD8281D002307F11B06F0
:103730009A4208D910F801CB06F801C001310133D3
:103740000529DBB2F4D103990A9104990B919342B4
:1037500007F11B010C9138BF043379680D9134BF18
:1037600055FA83F300230E93FB8AADF83EB0C3F302
:1037700009031A44069B8DF84230059B8DF84330AF
:1037800094F82C30ADF83C2083F001038DF84430E0
:1037900000238DF840A08DF841807B602A7BB88A99
:1037A000013A291DFFF76CF93B8BB882834203D1A4
:1037B000A3680AA92046984720460AA9FFF702FEF7
:1037C000FB7DBA8AC3F38403013303F01F039B021A
:1037D000FB823B8B9A420CBF00206FF01000C1E6C9
:1037E0007B68002BAFD0052001E01C3033461E68FB
:1037F000002EFAD1091A081D2E1D184401EB090CE0
:10380000BCF11B0F5FFA89F39DD89A429BD916F839
:10381000013B00F8013B09F10109EFE76FF00900F6
:10382000A0E66FF00A009DE66FF00B009AE66FF0DD
:103830000D0097E66FF00E0094E66FF00F0091E632
:1038400040420F0080841E00EFF3098305494A6B54
:1038500022F001024A63683383F30988002383F36B
:103860001188704700EF00E0302080F3118862B6C5
:103870000C4B0D4AD96821F4E0610904090C0A4394
:10388000DA60D3F8FC20094942F08072C3F8FC20CA
:103890000A6842F001020A602022DA7783F82200E7
:1038A000704700BF00ED00E00003FA05001000E0E3
:1038B00010B5302383F311880E4B5B6813F400635B
:1038C00014D0F1EE103AEFF30984683C4FF08073A6
:1038D000E361094BDB6B236684F3098800F0A4F8ED
:1038E00010B1064BA36110BD054BFBE783F31188B4
:1038F000F9E700BF00ED00E000EF00E0430600083C
:10390000460600084FF0E023002258684FF0FF31D0
:10391000930003F1604303F5614301329042C3F821
:103920008010C3F88011F3D27047000000F16043AB
:1039300003F561430901C9B283F80013012200F0C5
:103940001F039A4043099B0003F1604303F5614361
:10395000C3F880211A6070470023037582680369E9
:103960001B6899689142FBD25A68036042601060FC
:103970005860704700230375826803691B68996863
:103980009142FBD85A6803604260106058607047EB
:1039900008B50846302383F311880B7D032B05D02F
:1039A000042B0DD02BB983F3118808BD8B6900223D
:1039B0001A604FF0FF338361FFF7CEFF0023F2E779
:1039C000D1E9003213605A60F3E70000FFF7C4BF8B
:1039D000054BD9680875186802681A60536001229F
:1039E0000275D860FCF718BE003C002030B50C4BC7
:1039F000DD684B1C87B004460FD02B46094A684649
:103A000000F050F92046FFF7E3FF009B13B1684632
:103A100000F052F9A86907B030BDFFF7D9FFF9E708
:103A2000003C002091390008044B1A68DB6890685C
:103A30009B68984294BF002001207047003C002002
:103A4000084B10B51C68D86822681A6053600122C0
:103A50002275DC60FFF78EFF01462046BDE810406E
:103A6000FCF7DABD003C0020044B1A68DB68926862
:103A70009B689A4201D9FFF7E3BF7047003C0020E2
:103A800038B5074C074908480123002523706560B5
:103A900000F000FC0223237085F3118838BD00BFBD
:103AA000283E002028490008003C002008B572B6D6
:103AB000044B186500F0B6FA00F06EFB024B0322CF
:103AC0001A70FEE7003C0020283E002000F02AB9D2
:103AD000EFF3118020B9EFF30583302282F31188D0
:103AE0007047000010B530B9EFF30584C4F3080443
:103AF00014B180F3118810BDFFF7B6FF84F311886D
:103B0000F9E700008B60022308618B82084670474A
:103B10008368A3F1840243F8142C026943F8442C0F
:103B2000426943F8402C094A43F8242CC26843F800
:103B3000182C022203F80C2C002203F80B2C044A48
:103B400043F8102CA3F12000704700BF3106000895
:103B5000003C002008B5FFF7DBFFBDE80840FFF799
:103B600035BF0000024BDB6898610F20FFF730BFC4
:103B7000003C0020302383F31188FFF7F3BF0000DF
:103B800008B50146302383F311880820FFF72EFF84
:103B9000002383F3118808BD10B503689C68A24216
:103BA0000CD85C688A600B604C6021605960996831
:103BB0008A1A9A604FF0FF33836010BD1B68121B96
:103BC000ECE700000A2938BF0A2170B504460D460B
:103BD0000A26601900F058FB00F044FB041BA542C4
:103BE00003D8751C2E460446F3E70A2E04D9BDE817
:103BF0007040012000F08EBB70BD0000F8B5144B82
:103C00000D46D96103F1100141600A2A19698260E9
:103C100038BF0A22016048601861A818144600F0F5
:103C200025FB0A2700F01EFB431BA342064606D3D2
:103C30007C1C281900F028FB27463546F2E70A2F9E
:103C400004D9BDE8F840012000F064BBF8BD00BF16
:103C5000003C0020F8B506460D4600F003FB0F4A75
:103C6000134653F8107F9F4206D12A46014630463C
:103C7000BDE8F840FFF7C2BFD169BB68441A2C19F0
:103C800028BF2C46A34202D92946FFF79BFF2246B4
:103C900031460348BDE8F840FFF77EBF003C0020F6
:103CA000103C002010B4C0E9032300235DF8044B4E
:103CB0004361FFF7CFBF000010B5194C236998424C
:103CC0000DD0D0E90032816813605A609A680A44C6
:103CD0009A60002303604FF0FF33A36110BD2346B9
:103CE000026843F8102F53600022026022699A4252
:103CF00003D1BDE8104000F0C1BA936881680B445D
:103D0000936000F0AFFA2269E1699268441AA24216
:103D1000E4D91144BDE81040091AFFF753BF00BFB2
:103D2000003C00202DE9F047DFF8BC8008F11007C7
:103D30002C4ED8F8105000F095FAD8F81C40AA681C
:103D4000031B9A423ED81444D5E900324FF00009D3
:103D5000C8F81C4013605A60C5F80090D8F81030BD
:103D6000B34201D100F08AFA89F31188D5E9033111
:103D700028469847302383F311886B69002BD8D0ED
:103D800000F070FA6A69A0EB04094A4582460DD238
:103D9000022000F0BFFA0022D8F81030B34208D158
:103DA00051462846BDE8F047FFF728BF121A2244C3
:103DB000F2E712EB090938BF4A4629463846FFF7B1
:103DC000EBFEB5E7D8F81030B34208D01444211AFE
:103DD000C8F81C00A960BDE8F047FFF7F3BEBDE8D6
:103DE000F08700BF103C0020003C002000207047FE
:103DF000FEE70000704700004FF0FF307047000002
:103E0000BFF34F8F024A1369DB03FCD4704700BF36
:103E10000020024008B5094B1B7873B9FFF7F0FF8B
:103E2000074B5A69002ABFBF064A9A6002F18832DE
:103E30009A601A6822F480621A6008BD403E002031
:103E4000002002402301674508B50B4B1B7893B94E
:103E5000FFF7D6FF094B5A6942F000425A611A68CF
:103E600042F480521A601A6822F480521A601A686A
:103E700042F480621A6008BD403E002000200240EB
:103E80003F289ABF00F58030C00200207047000034
:103E90004FF4006070470000402070473F2808B58D
:103EA0000BD8FFF7EDFF00F500630268013204D183
:103EB00004308342F9D1012008BD0020FCE7000056
:103EC0003F2810B504461FD8FFF79AFFFFF7A2FF5F
:103ED0000E4BF3221A6102225A615A6942EAC00269
:103EE0005A615A6942F480325A61FFF789FF4FF4F0
:103EF0000061FFF7C5FF00F04BF9FFF7A5FF204673
:103F0000BDE81040FFF7CABF002010BD00200240EE
:103F10002DE9F84340EA020313F00703144606D0E4
:103F2000304B40F231321A600020BDE8F88385182A
:103F30002D4A95420CD92B4A40F236311160F3E7F5
:103F4000031D1B684A68934208D1083C08300831B9
:103F5000072C14D902680B689A42F1D0FFF75AFF78
:103F6000FFF74EFF214E08314FF001084FF00009D6
:103F7000012CA1F1080706D8FFF766FF01E0002C2D
:103F8000ECD10120D1E7C6F81480054651F8083C71
:103F900045F8043B51F8043C4360FFF731FF3369B7
:103FA00043F001033361C6F81490026851F8083CED
:103FB0009A420CD00B4B40F25E321A600C4B1860E8
:103FC0000C4B1C600C4B1F60FFF73EFFACE72D68ED
:103FD00051F8043C9D4201F10801EBD1083C083046
:103FE000C6E700BF3C3E002000000208002002405F
:103FF000303E0020383E0020343E0020084908B5FD
:104000000B7828B11BB9FFF705FF01230B7008BD22
:10401000002BFCD0BDE808400870FFF715BF00BFBB
:10402000403E002008B54FF4B0414FF0005000F082
:10403000B1F8BDE808404FF420514FF0805000F037
:10404000A9B80000084600F0E3BB000070B582B0DC
:10405000FFF73EFD0E4E054600F004F9326890422F
:1040600037BF0C4A0B49516814682EBFD1E9004193
:10407000013151600419034641F1000128460191C4
:104080003360FFF72FFD0199204602B070BD00BFDD
:10409000443E0020483E002070B582B0FFF718FD76
:1040A000104E054600F0DEF83268904237BF0E4AE7
:1040B0000D49516814682EBFD1E9004101315160AA
:1040C000041941F100010346284601913360FFF7CE
:1040D00009FD01994FF47A7200232046FCF788F815
:1040E00002B070BD443E0020483E00200244D2B2DF
:1040F000904200D17047431C800000F1804000F5E1
:104100001450006841F8040BD8B2F1E7124B10B517
:10411000D3F89040240409D4D3F89040C3F89040D9
:10412000D3F8904044F40044C3F890400B4C23680B
:10413000024443F480732360D2B2904200D110BD98
:10414000431C800000F1804000F5145051F8044BEE
:104150000460D8B2F1E700BF0010024000700040D8
:1041600007B5012201A90020FFF7C0FF019803B0A5
:104170005DF804FB13B50446FFF7F2FFA04205D03B
:10418000012201A900200194FFF7C0FF02B010BD79
:10419000704700007047000070470000074B45F271
:1041A00055521A6002225A6040F6FF729A604CF62D
:1041B000CC421A60024B01221A7070470030004056
:1041C000543E0020034B1B781BB1034B4AF6AA2236
:1041D0001A607047543E002000300040054B1A68BA
:1041E00032B902F1804202F50432D2F894201A600A
:1041F000704700BF503E0020024B4FF40002C3F84E
:10420000942070470010024008B5FFF7E7FF024B0B
:104210001868C0F3407008BD503E00207047000091
:10422000FEE700000A4B0B480B4A90420BD30B4BA6
:10423000DA1C121AC11E22F003028B4238BF002280
:104240000021FDF79FB853F8041B40F8041BECE76E
:104250008C4A0008D83E0020D83E0020D83E0020DE
:1042600000F0C2B84FF08043586A70474FF0804367
:10427000002258631A610222DA6070474FF08043CF
:104280000022DA60704700004FF0804358637047A7
:10429000FEE7000070B51B4B01630025044686B0A5
:1042A000586085620E46FFF7DFFA04F11003C4E997
:1042B00004334FF0FF33C4E90635C4E90044A56078
:1042C000E562FFF7CFFF2B460246C4E9082304F15D
:1042D00034010D4A256580232046FFF713FC012396
:1042E000E0600A4A0375009272680192B268CDE9F3
:1042F0000223074B6846CDE90435FFF72BFC06B0D7
:1043000070BD00BF283E002034490008394900082C
:1043100091420008024AD36A1843D062704700BF36
:10432000003C00204B6843608B688360CB68C360AF
:104330000B6943614B6903628B6943620B680360DD
:104340007047000008B5204BDA6A42F07F02DA625B
:10435000DA6A22F07F02DA62DA6ADA6C42F07F020D
:10436000DA64DA6E42F07F02DA66184ADB6E1146D2
:104370004FF09040FFF7D6FF02F11C0100F580607E
:10438000FFF7D0FF02F1380100F58060FFF7CAFFA8
:1043900002F1540100F58060FFF7C4FF02F17001E3
:1043A00000F58060FFF7BEFF02F18C0100F5806030
:1043B000FFF7B8FF02F1A80100F58060FFF7B2FF38
:1043C000BDE8084000F050B8001002404049000825
:1043D00008B500F0EDF9FFF753FBBDE80840FFF723
:1043E000FDBE0000704700000F4B9A6D42F00102C5
:1043F0009A659A6F42F001029A670C4A9B6F936824
:1044000043F0010393604FF08043A7229A624FF07C
:10441000FF32DA6200229A615A63DA605A6001223E
:104420005A611A60704700BF00100240002004E08B
:104430004FF0804208B51169D3680B40D9B2C94327
:104440009B07116107D5302383F31188FFF73EFBEB
:10445000002383F3118808BD08B5FFF753FABDE8C0
:10446000084000F081B900004E4B4FF0FF319A6ACE
:1044700099629A6A00229A62986AD86A60F07F000C
:10448000D862D86A00F07F00D862D86A186B1963C6
:10449000186B1A63186B986B9963986B9A63986B97
:1044A000D86BD963D86BDA63D86B186C1964196C44
:1044B0001A64196C196E41F001011966D3F8801065
:1044C00021F00101C3F88010D3F88010996D41F0FC
:1044D00080519965996F21F080519967996F3249A0
:1044E0004FF400408860CA600A624A628A62CA6207
:1044F0000A634A638A63CA630A644A648A64CA6450
:104500000A654A654A604FF48072C1F880204FF412
:1045100040720A604A6912F48062FBD1D3F89010AD
:1045200011F4407F1EBF4FF48031C3F89010C3F8E0
:104530009020D3F8982042F00102C3F89820D3F8D5
:1045400098209207FBD51A6842F480321A601A68E4
:104550009003FCD5D3F8902022F00322C3F89020DA
:10456000124ADA601A6842F080721A601A68910181
:10457000FCD50F490F4800229A60C3F888100E49F5
:10458000C3F89C20016002684A401207FBD19A6878
:1045900042F003029A609A6802F00C020C2AFAD1E7
:1045A000704700BF0010024000700040232A6101E4
:1045B000550100500020024004070400074A08B5D6
:1045C000536903F00103536123B1054A13680BB12A
:1045D00050689847BDE80840FFF76AB900040140F9
:1045E000583E0020074A08B5536903F0020353619F
:1045F00023B1054A93680BB1D0689847BDE80840DD
:10460000FFF756B900040140583E0020074A08B59C
:10461000536903F00403536123B1054A13690BB1D5
:1046200050699847BDE80840FFF742B900040140CF
:10463000583E0020074A08B5536903F00803536148
:1046400023B1054A93690BB1D0699847BDE808408A
:10465000FFF72EB900040140583E0020074A08B574
:10466000536903F01003536123B1054A136A0BB178
:10467000506A9847BDE80840FFF71AB900040140A6
:10468000583E0020164B10B55C6904F478725A61EC
:10469000A30604D5134A936A0BB1D06A9847600603
:1046A00004D5104A136B0BB1506B9847210604D503
:1046B0000C4A936B0BB1D06B9847E20504D5094ABD
:1046C000136C0BB1506C9847A30504D5054A936C45
:1046D0000BB1D06C9847BDE81040FFF7E9B800BFB8
:1046E00000040140583E0020194B10B55C6904F4E9
:1046F0007C425A61620504D5164A136D0BB1506DA8
:104700009847230504D5134A936D0BB1D06D984794
:10471000E00404D50F4A136E0BB1506E9847A10404
:1047200004D50C4A936E0BB1D06E9847620404D541
:10473000084A136F0BB1506F9847230404D5054AFC
:10474000936F0BB1D06F9847BDE81040FFF7B0B83A
:1047500000040140583E002008B5FFF769FEBDE89F
:104760000840FFF7A5B80000062108B50846FFF786
:10477000DDF806210720FFF7D9F806210820FFF70A
:10478000D5F806210920FFF7D1F806210A20FFF706
:10479000CDF806211720FFF7C9F806212820FFF7DA
:1047A000C5F8BDE8084007211C20FFF7BFB800008E
:1047B00008B5FFF751FE00F007F8FFF713FEBDE85C
:1047C0000840FFF74DBD00000023054A194601339C
:1047D000102BC2E9001102F10802F8D1704700BFA6
:1047E000583E00200B460146184600F003B8000072
:1047F00000F00EB810B5054C13462CB10A46014620
:104800000220AFF3008010BD2046FCE7000000004E
:10481000024B01461868FFF715BC00BF18110020B5
:1048200010B501390244904201D1002005E003781F
:1048300011F8014FA34201D0181B10BD0130F2E75F
:104840002DE9F041A3B1C91A17780144044603F1D8
:10485000FF3C8C42204601D9002009E00578BD428A
:1048600004F10104F5D10CEB0405D618A54201D1E1
:10487000BDE8F08115F8018D16F801EDF045F5D091
:10488000E7E70000034611F8012B03F8012B002A8B
:10489000F9D170476F72672E6172647570696C6FC1
:1048A000742E48697465632D41697273706565641F
:1048B0000000000040A2E4F1646891060041A3E515
:1048C000F2656992070000004261642043414E494D
:1048D0006661636520696E6465782E0000000000E3
:1048E000000000008D200008951B000849270008E3
:1048F0008D1B00083D1C0008211E0008051C000837
:10490000CD1B0008D11B0008A91B0008911B000843
:10491000E11D0008B51B000881280008C11B000824
:10492000B51D00086330000024490008583C0020F1
:10493000283E00206D61696E0069646C65000000AE
:104940000010802A00000000AAAAAAAA00000024E1
:10495000BFFF0000000000000090090000000001FF
:1049600000000000AAAAAAAA00000001FFFF0000A0
:104970000000000000000000000000000000000037
:10498000AAAAAAAA00000000FFFF00000000000081
:10499000000000000000000000000000AAAAAAAA6F
:1049A00000000000FFFF0000000000000000000009
:1049B0000000000000000000AAAAAAAA000000004F
:1049C000FFFF0000000000000000000000000000E9
:1049D00000000000AAAAAAAA00000000FFFF000031
:1049E00000000000000000000000000000000000C7
:1049F000AAAAAAAA00000000FFFF00000000000011
:104A0000000000001CB8FF7F010000000000000053
:104A100016040000000000000098010000000000E3
:104A2000FE2A0100D20400001C110020000000003A
:104A30000000000000000000000000000000000076
:104A40000000000000000000000000000000000066
:104A50000000000000000000000000000000000056
:104A60000000000000000000000000000000000046
:104A70000000000000000000000000000000000036
:0C4A80000000000000000000000000002A
:00000001FF
